:100000000C945B000C9427020C9454020C94830013
:100010000C9483000C9483000C9483000C94830054
:100020000C9483000C9483000C9483000C94830044
:100030000C9483000C9483000C9483000C94830034
:100040000C9481020C9483000C943D040C94830066
:100050000C9483000C9483000C9483000C94830014
:100060000C9483000C948300000024272A000025B0
:10007000282B000023262904040404040404040299
:100080000202020202030303030303010204081035
:100090002040800102040810200102040810200002
:1000A0000000070002010000030406000000000039
:1000B00000000000110211241FBECFEFD4E0DEBF0C
:1000C000CDBF11E0A0E0B1E0E0E1FCE002C00590AE
:1000D0000D92A231B107D9F711E0A2E1B1E001C060
:1000E0001D92A03FB107E1F710E0C6EBD0E004C0DD
:1000F0002297FE010E940206C43BD107C9F70E9465
:100100000A020C9406060C94000040E052EC61E0F8
:1001100070E08AE591E00E94220264E670E080E0EF
:1001200090E00E94F10261E0809100010E9463036F
:100130000895BF92CF92DF92EF92FF920F931F9399
:10014000DF93CF93CDB7DEB72A970FB6F894DEBF13
:100150000FBECDBF6B01DE011196E2E0F1E02AE0B7
:1001600001900D922150E1F79C0189589F4FFC01AD
:10017000849125573F4FF901B490E82FF0E0EE0F3E
:10018000FF1FEC0FFD1F0181128190E2E92EF12C7F
:10019000E00EF11EF80180A18B2980A38AE090E097
:1001A0000E941B03F894F80180A19B2D9095892350
:1001B00080A300000000000000000000000000001C
:1001C000000000000000000000000000000000002F
:1001D000000000000000000000000000000000001F
:1001E000000000000000000000000000000000000F
:1001F00000000000000000000000000000000000FF
:1002000000000000000000000000000000000000EE
:10021000000020E030E0C0FE04C0F70180818B299F
:1002200003C0F70180818923808300000000000063
:1002300000000000000000000000000000000000BE
:1002400000000000000000000000000000000000AE
:10025000000000000000000000000000000000009E
:10026000000000000000000000000000000000008E
:10027000000000000000000000000000000000007E
:10028000000000000000000000002F5F3F4F2830FA
:10029000310519F0D594C794BECFF80180A18B2900
:1002A00080A378942A960FB6F894DEBF0FBECDBF18
:1002B000CF91DF911F910F91FF90EF90DF90CF9042
:1002C000BF900895CF93DF9360E0809100010E947A
:1002D00081036AE070E080E090E00E94F1021092F9
:1002E0001A01C0E0D0E08091000190910101C0347A
:1002F000D10531F0FE01E65EFE4F608170E002C084
:100300006FEF70E00E9499002196C134D10559F732
:10031000DF91CF9108958AE591E00E941F02882322
:1003200009F469C08091120190911301893C9105F3
:100330000CF459C0893D9105C1F48AE591E00E9411
:100340001C02AA2797FDA095BA2FBC01CD010E94DF
:10035000AD042AE939E949E95FE30E9439050E94C1
:100360007A047093150160931401809112019091A9
:1003700013018A3D9105C1F48AE591E00E941C02B7
:10038000AA2797FDA095BA2FBC01CD010E94AD040C
:100390002AE939E949E95FE30E9439050E947A04B4
:1003A00070931701609316018091120190911301CF
:1003B0008B3D9105C1F48AE591E00E941C02AA27B9
:1003C00097FDA095BA2FBC01CD010E94AD042AE98A
:1003D00039E949E95FE30E9439050E947A04709384
:1003E0001901609318018AE591E00E941C02909324
:1003F0001301809312018091140180932101809157
:1004000016018093220180911801809323010E949C
:10041000620108950E9429030E9485000E948B01B9
:10042000FDCF80E191E090935B0180935A010895A4
:10043000862F0E94050408950E941E0408950E94BC
:100440000D040895CB01BA010E94CC0308951F92B8
:100450000F920FB60F9211242F933F934F935F93F8
:100460006F937F938F939F93AF93BF93EF93FF937C
:1004700080915C0190915D01892B29F0E0915C01F4
:10048000F0915D010995FF91EF91BF91AF919F911F
:100490008F917F916F915F914F913F912F910F902D
:1004A0000FBE0F901F9018951F920F920FB60F92CC
:1004B00011242F933F934F935F936F937F938F9369
:1004C0009F93AF93BF93EF93FF9380915E019091C1
:1004D0005F01892B29F0E0915E01F0915F010995A0
:1004E000FF91EF91BF91AF919F918F917F916F910C
:1004F0005F914F913F912F910F900FBE0F901F90E2
:1005000018951F920F920FB60F9211242F938F936D
:100510009F93AF93BF938091600190916101A091EF
:100520006201B09163010196A11DB11D809360012C
:1005300090936101A0936201B09363018091640183
:1005400090916501A0916601B09167018050904C37
:10055000AF4FBF4F8093640190936501A0936601F4
:10056000B093670127C08091640190916501A091CB
:100570006601B091670180589E43A040B0408093CF
:10058000640190936501A0936601B0936701809127
:10059000680190916901A0916A01B0916B01019687
:1005A000A11DB11D8093680190936901A0936A0118
:1005B000B0936B018091640190916501A0916601F7
:1005C000B091670181589E43A040B04060F6BF9152
:1005D000AF919F918F912F910F900FBE0F901F9011
:1005E0001895EF92FF920F931F937B018C018FB7A9
:1005F000F894409168015091690160916A0170918D
:100600006B018FBF2FB7F8948091680190916901B9
:10061000A0916A01B0916B012FBF841B950BA60BB3
:10062000B70BE816F9060A071B0760F71F910F9131
:10063000FF90EF900895019759F0FC01EE0FFF1F16
:10064000EE0FFF1F32978FB7F8943197F1F78FBFF6
:100650000895789484B5826084BD84B5816084BD3A
:1006600085B5826085BD85B5816085BDEEE6F0E02B
:10067000808181608083E1E8F0E080818260808316
:10068000808181608083E0E8F0E080818160808308
:10069000E1EBF0E0808184608083E0EBF0E080813A
:1006A00081608083EAE7F0E08081846080838081DC
:1006B0008260808380818160808380818068808384
:1006C0001092C1000895282F30E0C90185579F4F2F
:1006D000FC01949129583F4FF9018491882381F0BE
:1006E000E82FF0E0E859FF4FE491F0E0662329F4A9
:1006F000808190958923808308958081892B8083D0
:100700000895482F50E0CA0181569F4FFC01249163
:10071000CA0185579F4FFC01949149585F4FFA01D8
:1007200034913323C1F1222331F1233021F480911C
:1007300080008F7705C0243031F4809180008F7D58
:100740008093800018C0213019F484B58F7704C0DD
:10075000223021F484B58F7D84BD0DC0263021F474
:100760008091B0008F7705C0273029F48091B000C8
:100770008F7D8093B000E32FF0E0E359FF4FE491C9
:10078000F0E0662329F48081909589238083089581
:100790008081892B80830895EF92FF920F931F939E
:1007A0007B018C0122E030E040E050E00E94D10566
:1007B000205C3D4B404F5F4FCA01B901A801970132
:1007C0000E94D105C901DA010197A109B109292FB8
:1007D0003A2F4B2F552747FD5A950196A11DB11D64
:1007E0002093C50081508093C400E1ECF0E080814B
:1007F000806180838081886080838081806880833D
:100800001F910F91FF90EF900895982F8091C00055
:1008100085FFFCCF9093C600089580916C01909164
:100820006D0180589F4F20916E0130916F01821BA6
:10083000930B60E870E00E949C05089540916E0162
:1008400050916F0180916C0190916D018417950713
:1008500019F42FEF3FEF0FC0FA01E059FE4F20814E
:10086000CA01019660E870E00E949C0590936F01B8
:1008700080936E0130E0C90108951F920F920FB668
:100880000F9211242F933F934F935F936F937F9316
:100890008F939F93AF93BF93EF93FF934091C600C5
:1008A000E0916C01F0916D01CF01019660E870E07C
:1008B0000E949C059C0180916E0190916F01281708
:1008C000390739F0E059FE4F408330936D01209392
:1008D0006C01FF91EF91BF91AF919F918F917F91AB
:1008E0006F915F914F913F912F910F900FBE0F909D
:1008F0001F90189504D06894B111B5C0089598D090
:1009000088F09F5790F0B92F9927B751A0F0D1F0F8
:10091000660F771F881F991F1AF0BA95C9F712C082
:10092000B13081F09FD0B1E008959CC0672F782F3F
:100930008827B85F39F0B93FCCF3869577956795EE
:10094000B395D9F73EF490958095709561957F4F5A
:100950008F4F9F4F0895E89409C097FB3EF4909500
:100960008095709561957F4F8F4F9F4F9923A9F088
:10097000F92F96E9BB279395F69587957795679517
:10098000B795F111F8CFFAF4BB0F11F460FF1BC05B
:100990006F5F7F4F8F4F9F4F16C0882311F096E9EE
:1009A00011C0772321F09EE8872F762F05C066239C
:1009B00071F096E8862F70E060E02AF09A95660F55
:1009C000771F881FDAF7880F9695879597F908950E
:1009D00097F99F6780E870E060E008959FEF80ECF2
:1009E000089500240A941616170618060906089595
:1009F00000240A9412161306140605060895092EFB
:100A00000394000C11F4882352F0BB0F40F4BF2B69
:100A100011F460FF04C06F5F7F4F8F4F9F4F0895A9
:100A200057FD9058440F551F59F05F3F71F047959F
:100A3000880F97FB991F61F09F3F79F08795089584
:100A4000121613061406551FF2CF4695F1DF08C0A3
:100A5000161617061806991FF1CF869571056105C0
:100A600008940895E894BB2766277727CB0197F968
:100A700008950BD0C4CFB5DF28F0BADF18F0952366
:100A800009F0A6CFABCF1124EECFCADFA0F3959F1C
:100A9000D1F3950F50E0551F629FF001729FBB2765
:100AA000F00DB11D639FAA27F00DB11DAA1F649F11
:100AB0006627B00DA11D661F829F2227B00DA11DC4
:100AC000621F739FB00DA11D621F839FA00D611D4A
:100AD000221F749F3327A00D611D231F849F600D6B
:100AE000211D822F762F6A2F11249F5750408AF0A4
:100AF000E1F088234AF0EE0FFF1FBB1F661F771F30
:100B0000881F91505040A9F79E3F510570F060CF6B
:100B1000AACF5F3FECF3983EDCF386957795679517
:100B2000B795F795E7959F5FC1F7FE2B880F911D4D
:100B30009695879597F9089597FB092E07260AD071
:100B400077FD04D049D006D000201AF47095619545
:100B50007F4F0895F6F7909581959F4F0895A1E2F4
:100B60001A2EAA1BBB1BFD010DC0AA1FBB1FEE1F27
:100B7000FF1FA217B307E407F50720F0A21BB30B72
:100B8000E40BF50B661F771F881F991F1A9469F7EE
:100B900060957095809590959B01AC01BD01CF014A
:100BA000089597FB092E05260ED057FD04D0D7DFF8
:100BB0000AD0001C38F450954095309521953F4F50
:100BC0004F4F5F4F0895F6F790958095709561951A
:100BD0007F4F8F4F9F4F0895AA1BBB1B51E107C04A
:100BE000AA1FBB1FA617B70710F0A61BB70B881FBD
:100BF000991F5A95A9F780959095BC01CD0108954C
:100C0000EE0FFF1F0590F491E02D0994F894FFCFAB
:100C1000050000000000050008000B0000000000B7
:020C20001802B8
:00000001FF
